:020000040000FA
:02000000422894
:080008009C00030E9D00831211
:100010000B1918288B1811281D0E83009C0E1C0E1E
:1000200009000630980080309A000B128B100728C8
:100030009303190B2528951C30281F089B00283096
:1000400099009510031006172C2899000339031DF9
:100050003028061703149B0C031C061303180617FD
:100060000B1E980B3E2804309800060C9A0C031CBB
:100070003E281A089E0015158B100B169B30810721
:100080000B110C28960197019501900183168601AA
:1000900006148501CF30810001138312850186018A
:1000A0000130990098019B308100B0308B00951190
:1000B0001512861497010230960015110530920032
:1000C000FF309100930803199103930803199303D8
:1000D000910803197128151D62281511960B6028C7
:1000E00077289103920392080319572860289012E9
:1000F000A4211708031D90161010A4211708031D32
:100100001014A0009010A4211708031D9014A10042
:10011000A4211708A200951AA4219512A42117085A
:10012000A300A4211708A400A4211708A500FE30ED
:100130008C008D008E008F00152217088C00151A78
:10014000CC28152217088D00151ACC28152217085F
:100150008E00151ACC28152217088F00151ACC28E6
:1001600002309200FF309100930803199103930825
:100170000319930391080319C028151DB428C52835
:10018000920392080319CB28B22815111E080D3AC4
:10019000031DB228CC28951524298610861606152D
:1001A00015109E219E2100309F2110309400502276
:1001B000003A031D00003C22A7003C22A6003C227E
:1001C00000003C22103094005022003A031D000031
:1001D0003C22A7003C22A6003C2200003C22173013
:1001E00094005022003A031D00003C22A9003C224A
:1001F000A8003C2200003C22183094005022003A13
:10020000031D00003C22AB003C22AA003C2200005F
:100210003C22123094005022003A031D00003C2280
:10022000AD003C22AC003C2200003C221A3094007D
:100230005022003A031D00003C22AF003C22AE00D9
:100240003C2200003C22061186176B22951D3429A2
:100250009001A001A101A201A301A401A501FE300A
:100260008C008D008E008F009E2147309F21220838
:100270009F219E2147309F2122089F219E214830A7
:100280009F2123089F219E2149309F2124089F21DF
:100290009E214A309F2125089F219E214B309F217E
:1002A00020089F219E214C309F2121089F219E21C3
:1002B0004D309F210C089F219E214E309F210D081B
:1002C0009F219E214F309F210E089F219E2150305B
:1002D0009F210F089F219E2151309F2110089F21AF
:1002E000992981309F2151309F2126089F2127087D
:1002F0009F2181309F2153309F2128089F21290869
:100300009F2181309F2155309F212A089F212B0852
:100310009F2181309F2157309F212C089F212D083C
:100320009F2181309F2159309F212E089F212F0826
:100330009F21000095189A29861357288030951818
:100340009F299F0095140800FF3097009519080019
:1003500091009308031991039308031993039108DB
:100360000319122A151DA92915111E083B3A031954
:1003700008001E082D3A031DC02997019516080094
:1003800030301E029700FF3091009308031991034B
:1003900093080319930391080319122A151DC529FF
:1003A00015111E083B3A031908001708170717070D
:1003B00017071707170717071707170717079700D4
:1003C00030301E029707FF30910093080319910304
:1003D00093080319930391080319122A151DE5299F
:1003E00015111E083B3A03190800170817071707CD
:1003F0001707170717071707170717071707970094
:1004000030301E029707FF309100930803199103C3
:1004100093080319930391080319122A151D052A3D
:100420001511080015119515080095190800FF30E1
:1004300091009308031991039308031993039108FA
:100440000319362A151D192A1E082C3A0319322AB7
:100450001E080D3A0319392A1E0830301E02970073
:1004600015110800FF30970015110800151195159A
:1004700008001511151608001518003432309100C7
:10048000930803199103930803199303910803191F
:100490004E2A151D402A15111E0808001514003497
:1004A00015119E219E219E2100309F2101309F2108
:1004B00001309F2114089F211408023E9F213C22F5
:1004C0003C223C223C220000033A031D08003C224F
:1004D0003C223C22003432309100930803199103EE
:0E04E0009308031993039108031908006D2A6D
:00000001FF
